:100000000C942C030C9454030C9454030C9454033C
:100010000C9454030C9454030C9454030C94540304
:100020000C9454030C9454030C94772E0C941A2DB6
:100030000C9454030C9454030C9454030C945403E4
:100040000C9454030C9454030C9454030C945403D4
:100050000C94D30C0C9454030C9454030C946A0326
:100060000C9454030C9454030C9454030C945403B4
:100070000C9454030C9454030C9454030C945403A4
:100080000C9454030C9454030C9454030C94540394
:100090000C9454030C9454030C9454030C94540384
:1000A0000C9454030C9454030C9454036C6F6361CC
:1000B0006C6C79206275696C74206F6E204A756C67
:1000C00020323820323032322061742030373A32D8
:1000D000313A3032004B6579626F617264696F202A
:1000E000417472657573202D204B616C6569646F76
:1000F00073636F7065200014001A00080015001764
:1001000000000000001C0018000C00120013000486
:10011000001600070009000A00000000000B000D97
:10012000000E000F0033001D001B00060019000523
:10013000003500310011001000360037003800296A
:10014000002B00E300E1002A00E000E2002C002B7D
:10015000442D00340028001E081F085200210822E8
:1001600008000000004B002400250026002A00267D
:1001700008500051004F002708000000004E0021E9
:100180000022002300FFFF2F00300020082F08303E
:10019000082308240825081E001F0020002E08023E
:1001A000444900E300E1004C00E000E2002C00FFC5
:1001B000FF370027002E0049004A0052004D004B37
:1001C0000000000000520040004100420043004C8B
:1001D00000500051004F004E000000000051003D53
:1001E000003E003F0044000160E94800000000FFBD
:1001F000FFFFFFFFFF00003A003B003C00450054BA
:1002000044EA48FFFFFFFFFFFFFFFFFFFFFFFF5430
:100210004446004700CD48302E31312E302B323746
:100220000076657273696F6E0076657273696F6EC2
:100230000005010906A101050719E029E7150025B8
:100240000175019508810295017508810195057573
:100250000105081901290591029501750391019580
:10026000067508150025FF0507190029FF8100C044
:10027000050C0901A1018504150026FF0319002AB8
:10028000FF03950475108100C005010906A10185D1
:1002900008050719E029E715002501750195088172
:1002A00002050819012908950875019102050775CD
:1002B0000495018101190429DD15002501750195B9
:1002C000D98102750395018101C005010980A10151
:1002D0008505150026FF00190029FF950175088185
:1002E00000C0656570726F6D2E6572617365006523
:1002F0006570726F6D2E6672656500656570726FF0
:100300006D2E636F6E74656E747300656570726FC9
:100310006D2E636F6E74656E74730A656570726FAF
:100320006D2E667265650A656570726F6D2E6572F9
:10033000617365002F006372630076657273696F85
:100340006E0076616C69643F0064656661756C740B
:100350004C617965720073657474696E67732E0001
:1003600073657474696E67732E64656661756C7409
:100370004C617965720A73657474696E67732E7661
:10038000616C69643F0A73657474696E67732E7675
:10039000657273696F6E0A73657474696E67732E24
:1003A00063726300637573746F6D00646566617575
:1003B0006C74006F6E6C79437573746F6D006B6550
:1003C000796D61702E006B65796D61702E63757348
:1003D000746F6D0A6B65796D61702E646566617509
:1003E0006C740A6B65796D61702E6F6E6C794375F4
:1003F00073746F6D00454550524F4D4B65796D617B
:1004000070006573636170655F6F6E6573686F74AC
:100410002E63616E63656C5F6B6579006573636104
:1004200070655F6F6E6573686F742E63616E636570
:100430006C5F6B6579004573636170654F6E6553E2
:10044000686F740066616C73650074727565007026
:100450006C7567696E73006465766963652E726595
:100460007365740068656C700A6465766963652EEF
:1004700072657365740A706C7567696E7300686580
:100480006C70000D0A2E004D6163726F73001E08C0
:1004900034082008210822082408340026082708E8
:1004A00025082E0836002D003700380027003308B5
:1004B000330036082E00370838081F082F00310097
:1004C000300023082D0835002F0831083008350882
:1004D0004D6F7573654B657973004F6E6553686F2B
:1004E000740051756B657973005370616365436186
:1004F0006465740074726967676572006D6170008D
:100500006D6163726F732E006D6163726F732E6D18
:1005100061700A6D6163726F732E747269676765CB
:10052000720044796E616D69634D6163726F73002F
:1005300073697A653D006B65796D61702E6C6179C8
:1005400065724E616D6573006B65796D61702E6CBF
:10055000617965724E616D6573004C617965724EAB
:10056000616D657300080B000202020000090400BF
:100570000001020200000524001001052401010110
:10058000042402060524060001070581031000402B
:1005900009040100020A00000007050202400000F1
:1005A0000705830240000012010002EF020140092A
:1005B0001203230001010203014B6579626F61722E
:1005C00064696F0041747265757300040309040562
:1005D000010902A101850105091901290815002554
:1005E00001950875018102050109300931093815A5
:1005F00081257F750895038106050C0A380215814F
:10060000257F750895018106C005010902A1010534
:1006100009190129081500250195087501810205B0
:10062000010930093116000026FF7F7510950281FF
:100630000209381581257F750895018106C0A40C33
:10064000720E0B0FFF0F5E109411CE1586219023B2
:1006500036281F2FFA30CE3111241FBECFEFDAE03B
:10066000DEBFCDBF11E0A0E0B1E0EAE6F5E602C0F2
:1006700005900D92A63AB107D9F724E0A6EAB1E0B9
:1006800001C01D92AE3EB207E1F713E0CCE2D3E029
:1006900004C02197FE010E941D32CF31D107C9F756
:1006A0000E9457030C94B3320C94000008950E94EA
:1006B00029040E9456038EE394E00E94EF2E0E94CC
:1006C0006305C0E0D0E00E9480052097E1F30E941E
:1006D0000000F9CF1F920F920FB60F9211242F93A3
:1006E0003F938F939F93AF93BF938091A701909176
:1006F000A801A091A901B091AA013091A60123E01F
:10070000230F2D3758F50196A11DB11D2093A60189
:100710008093A7019093A801A093A901B093AA0187
:100720008091AB019091AC01A091AD01B091AE016F
:100730000196A11DB11D8093AB019093AC01A093D4
:10074000AD01B093AE01BF91AF919F918F913F9159
:100750002F910F900FBE0F901F90189526E8230F32
:100760000296A11DB11DD2CF2FB7F8946091A701B9
:100770007091A8018091A9019091AA012FBF0895BD
:100780003FB7F8948091AB019091AC01A091AD017D
:10079000B091AE0126B5A89B05C02F3F19F0019678
:1007A000A11DB11D3FBFBA2FA92F982F8827BC01CB
:1007B000CD01620F711D811D911D42E0660F771FF3
:1007C000881F991F4A95D1F708958F929F92AF92F3
:1007D000BF92CF92DF92EF92FF926B017C010E9459
:1007E000C0034B015C01C114D104E104F104E9F040
:1007F0000E941E2F0E94C003681979098A099B096B
:10080000683E73408105910570F321E0C21AD1085A
:10081000E108F10888EE880E83E0981EA11CB11C47
:10082000C114D104E104F10429F7FF90EF90DF90A7
:10083000CF90BF90AF909F908F9008958230910598
:1008400038F0880F991F880F991F05970197F1F7C6
:100850000895789484B5826084BD84B5816084BD38
:1008600085B5826085BD85B5816085BDEEE6F0E029
:10087000808181608083E1E8F0E010828081826085
:100880008083808181608083E0E8F0E08081816006
:100890008083E1E9F0E080818260808380818160F3
:1008A0008083E0E9F0E0808181608083E1ECF0E02A
:1008B0008081846080838081826080838081816088
:1008C0008083E3ECF0E0808181608083E0ECF0E005
:1008D000808182608083E2ECF0E0808181608083AF
:1008E000EAE7F0E080818460808380818260808399
:1008F00080818160808380818068808308950895ED
:1009000086E0ECE4F1E0DB0101900D928A95E1F7DD
:1009100086E0089583EE92E00E943C1381E393E029
:100920000E94471E87E693E00E94FB2182E191E04E
:100930000E94D41C8BE093E00E949C1788E993E00E
:100940000E943C258CE193E00E94991888EE92E089
:100950000E94E9148DED93E00C94122689ED92E04B
:100960000E948F1083EE92E00E9432138CE193E09C
:100970000E94AE1888EE92E00E94A91480E00895CB
:1009800089ED92E00E948C1180E00895CF93DF936F
:10099000EC01BC0181E393E00E94D720811107C0E4
:1009A000BE0187E693E0DF91CF910C941823DF918D
:1009B000CF910895CF93DF93EC01BC0185E091E0E6
:1009C0000E94521581111CC0BE0182E191E00E947B
:1009D0008A1D811115C0BE018BE093E00E9464174F
:1009E00081110EC0BE0188E993E00E941925811192
:1009F00007C0BE018CE193E0DF91CF910C942419E4
:100A0000DF91CF910895BC018CE193E00C94DE1846
:100A100080E00895CF93DF93EC01BC018CE093E07C
:100A20000E947A18811107C0BE018CE093E0DF912B
:100A3000CF910C947A18DF91CF910895CF93DF93E3
:100A4000EC01BC0182E191E00E94781DBE018CE1C5
:100A500093E00E94E01980E0DF91CF9108958AEE43
:100A600092E00E94D11581E393E00E94482187E63D
:100A700093E00E94B62282E191E00E94E91C8CE1A1
:100A800093E00E94981980E00895FB01918191FF05
:100A900006C090FD04C0882329F0813039F090E031
:100AA00080E0089580E00E94B40BF9CF65ED70E01E
:100AB0008BE093E00E9445176CEA70E08BE093E0D6
:100AC0000E944517ECCF80915301909154010E94F0
:100AD000A00A81E08093670389E00E945C1360E3D1
:100AE00070E088E993E00E9451256FE370E08DED9E
:100AF00093E00E9423268091DD028F770C94B40B43
:100B000080915301909154010C94530B0F931F93B8
:100B1000CF93DF93EC016881798183EE92E00E94AC
:100B2000DE13811157C0688179818AEE92E00E94BC
:100B3000931581114FC06881798187ED92E00E9401
:100B4000AA11811147C06881798188ED92E00E94E5
:100B50003A1281113FC06881798188E993E00E944F
:100B60006A25811137C06881798188EE92E00E9400
:100B7000FE1481112FC00881198149E252E0B801A9
:100B80008AEE92E00E947E1581111AC061E272E045
:100B9000C8010E945E32892B99F467E172E081EE10
:100BA00093E00E94362984E690E00E941E0460E2F1
:100BB00081EE93E00E945A2984E690E00E941E0490
:100BC000688179818DED93E0DF91CF911F910F9135
:100BD0000C943626DF91CF911F910F910895CF93FA
:100BE000DF9300D0CDB7DEB79A838983CE0101961B
:100BF0000E9486050F900F90DF91CF91089581E4B8
:100C000092E00E945B0E80E892E00E94F50F82E67F
:100C100092E00E94090F88EC92E00C944210E5E506
:100C2000F1E050E040E070E060E000009191A92F19
:100C3000B0E084E0B595A7958A95E1F790962C9160
:100C400030E09F7002C0359527959A95E2F7209580
:100C5000309521703327042E02C0220F331F0A94CF
:100C6000E2F7622B732B4F5F5F4F4C305105E9F673
:100C7000CB0108951F93CF93DF93C1E1D2E010E041
:100C8000288139818A819B81482F440F4270522FDD
:100C90005170452B09F005C1AC0156954795440F9D
:100CA000427021FB552750F9452B09F0EFC0AC01EC
:100CB0005695479556954795440F427022FB552708
:100CC00050F9452B09F0D7C0AC015695479556957C
:100CD000479556954795440F427023FB552750F989
:100CE000452B09F0BDC0AC01529542954F70452788
:100CF0005F704527440F427024FB552750F9452B60
:100D000009F0A3C0AC0156954795529542954F7096
:100D100045275F704527440F427025FB552750F942
:100D2000452B09F087C0AC010024440F551F001C5F
:100D3000440F551F001C452F502D440F427026FBB9
:100D4000552750F9452B09F06AC0AC01440F452FD7
:100D5000441F550B5195440F427027FB222720F961
:100D6000422B09F052C0492F440F4270232F2170AB
:100D7000422B09F040C031FB222720F9492F427055
:100D8000422B79F5492F4695427032FB222720F9F4
:100D9000422BE9F4292F26952695227033FB442710
:100DA00040F9422B59F4998388832A96145F1033B3
:100DB00009F066CFDF91CF911F9108956BE0610F2D
:100DC00080E090E00E94A70C8A819B81ECCF6AE0D2
:100DD000610F80E090E00E94A70C39818A819B819D
:100DE000D9CF69E0610F80E090E00E94A70C3981C3
:100DF0008A819B81C7CF68E0610F80E090E00E940C
:100E0000A70C39818A819B81B6CF67E0610F80E0B2
:100E100090E00E94A70C39818A819B81A4CF66E073
:100E2000610F80E090E00E94A70C288139818A81BF
:100E30009B818BCF65E0610F80E090E00E94A70C62
:100E4000288139818A819B816ECF64E0610F80E0C7
:100E500090E00E94A70C288139818A819B8152CF22
:100E600063E0610F80E090E00E94A70C2881398147
:100E70008A819B8138CF62E0610F80E090E00E9420
:100E8000A70C288139818A819B811ECF61E0610F87
:100E900080E090E00E94A70C288139818A819B81A3
:100EA00006CF612F80E090E00E94A70C2881398155
:100EB0008A819B81F1CE81E492E00E94B60D81117E
:100EC00004C081E492E00C94B90D80E892E00E94A5
:100ED0003B0F82E692E00C94E30E81E492E00E94E4
:100EE000B60D811104C081E492E00C94540E80E8A8
:100EF00092E00E94EF0F82E692E00C94D00ECF9326
:100F0000C82F81E492E00E94B60D6C2F811105C0BC
:100F100081E492E0CF910C941C0E80E892E0CF9196
:100F20000C94C60FCF93C82F81E492E00E94B60DB7
:100F30006C2F811105C081E492E0CF910C94F50DE6
:100F400080E892E0CF910C949F0FCF93C82F83FF3E
:100F500003C081EE0E949207C0FF03C080EE0E9492
:100F60009207C1FF03C082EE0E949207C2FF03C036
:100F700086EE0E949207C4FF04C083EECF910C94CA
:100F80009207CF910895CF93C82F892F0E94A5076C
:100F90008C2FCF910C949207FC019081DB018C91F6
:100FA000981305C081E0218111969C91291380E05E
:100FB00008951F93CF93DF9300D000D0CDB7DEB755
:100FC000182F803368F5E82FF0E0EE0FFF1FE75B86
:100FD000FB4F808191819C838B838FEF89838A83F0
:100FE000BE016F5F7F4FCE0103960E94CC0788231E
:100FF00069F0A12FB0E0AB54BE4FE0910201F09137
:101000000301612F8C9109958B839C838B819C813B
:101010000F900F900F900F90DF91CF911F91089537
:101020001092A9041092AA04E9EAF4E0D2CF1F9327
:10103000CF93DF93C62F172F862F972F0E9403057C
:10104000823009F1812F807C61F480E28C0F88303E
:1010500008F010E08C2F912FDF91CF911F910C940D
:10106000C307812F887C883471F4612F70E0762F5C
:1010700066276C0F711D737082E692E0DF91CF914D
:101080001F910C94BB0EDF91CF911F9108958F9209
:101090009F92BF92CF92DF92EF92FF920F931F9396
:1010A000CF93DF9300D000D000D0CDB7DEB77C0166
:1010B0006B010E946D0710E000E0BB24BA9400337E
:1010C000110599F1F6019081901729F1003330F55F
:1010D000F801EE0FFF1FE75BFB4F808091809E823F
:1010E0008D82BB82BC82BE016D5F7F4FCE010596B3
:1010F0000E94CC0781110FC019821A82BE016F5F56
:101100007F4FCE0105960E94CC07811104C0B40127
:10111000C7010E9417080F5F1F4FD1CF1092A9047B
:101120001092AA04E9EAF4E0D8CF26960FB6F89414
:10113000DEBF0FBECDBFDF91CF911F910F91FF900A
:10114000EF90DF90CF90BF909F908F900895EF9297
:10115000FF920F931F93CF93DF938C01EB01898153
:1011600081FF43C080FD41C08B81807CF1F5888187
:1011700080930101FA8081E492E00E94B60D6F2D08
:1011800081112EC081E492E00E94650E882301F156
:10119000FB80EA80F3FE03C081EE0E947F07F0FE31
:1011A00003C080EE0E947F07F1FE03C082EE0E9422
:1011B0007F07F2FE03C086EE0E947F07F4FE03C0A5
:1011C00083EE0E947F078E2D0E947F070E945B079F
:1011D0008B81882379F00E94A5070E945B070AC0D3
:1011E00080E892E00E94890FD1CFE09101018881CF
:1011F000E81317C0898181FF07C080FD05C06A819F
:101200007B81C8010E941708CE010E940A05823026
:10121000E9F0DF91CF911F910F91FF90EF900C9427
:101220005B07E03360F4F0E0EE0FFF1FE75BFB4F7E
:101230008181982F907CF1F60E94A507DBCF109258
:10124000A9041092AA04E9EAF4E0F2CFDF91CF9169
:101250001F910F91FF90EF900895FF920F931F93AE
:10126000CF93DF93CDB7DEB72D970FB6F894DEBFDF
:101270000FBECDBF8C0129873A874B875C876D876E
:10128000203348F430FF61C031FD5FC089850E9482
:10129000D9079C878B87CE0109960E94DA04823099
:1012A00009F447C0E985E03368F49A85F0E0EE0F71
:1012B000FF1FE75BFB4F90FF55C091FD53C09FEFB1
:1012C00090839183811135C01F821886BE01695FAA
:1012D0007F4FCE010B960E94CC0781112AC01D8240
:1012E0001E82BE016B5F7F4FCE010B960E94CC0722
:1012F00081111FC0FF24FA94FB82FC82BE016D5F46
:101300007F4FCE010B960E94CC07811112C0F9824B
:10131000FA82BE016F5F7F4FCE010B960E94CC0711
:10132000811107C08C85843409F5CE0109960E948D
:10133000450C2D960FB6F894DEBF0FBECDBFDF91E2
:10134000CF911F910F91FF9008958FEF89838A832A
:10135000BE016F5F7F4FCE010B960E94CC078111BB
:1013600095CF99CF9C852B852083ABCF8F7C813403
:10137000B9F48A851B8581FF0AC080FD08C0612FF2
:1013800088EC92E00E94461010930902D2CF80911F
:1013900009028113CECF88EC92E00E944410C9CF9D
:1013A000BE01675F7F4FC8010E944708BE01675FAB
:1013B0007F4FC8010E94A708CE0109960E941E0512
:1013C000B8CFEF92FF920F931F93CF93DF9300D08C
:1013D00000D000D01F92CDB7DEB7022F2B833C8305
:1013E0004D835E836F83203308F042C07C01832FDE
:1013F000817031FF22C081113BC08FEF89838A83C6
:10140000BE016F5F7F4FCE0105960E94CC078823F7
:1014100029F0802F0E94D9079E838D83CE010396E9
:101420000E94C604811124C02B813C814D815E81C4
:101430006F81C7010E942D091BC08823C9F010E0ED
:10144000000F111F075B1B4FF801808191819E8364
:101450008D8319821A82BE016F5F7F4FCE01059680
:101460000E94CC078823D1F28FEFF801808381831B
:1014700027960FB6F894DEBF0FBECDBFDF91CF9198
:101480001F910F91FF90EF900895CF930FB6F894AE
:10149000A895809160008861809360001092600040
:1014A0000FBEA5E5B1E041E651E061E070E08D914D
:1014B000E82FF0E024E0F595E7952A95E1F7C1A142
:1014C0008F709B0101C0220F8A95EAF7922F9095A9
:1014D0009C2391A382A1822B82A34A175B0739F731
:1014E000A1E6B1E045E651E061E070E08D91E82FC2
:1014F000F0E094E0F595E7959A95E1F791A18F706A
:101500009B0101C0220F8A95EAF7922B91A382A139
:10151000822B82A34A175B0749F780E18093810001
:101520001092800080EE9EE2909387008093860068
:1015300081E18093810081E080936F00CF910895D5
:101540000E94FF058CE092E00E94450A40E855E2C7
:1015500060E070E081EE93E00E9430280E947F04FA
:101560000E94AE04E9E4F4E081E39FEF815021F0B2
:10157000908391833296FACF84EB91E00C94B20B76
:101580006F927F928F929F92AF92BF92CF92DF9293
:10159000EF92FF920F931F93CF93DF9321E6E22EFA
:1015A00021E0F22EC1E1D2E035E6632E31E0732E68
:1015B000912C812CAA24A394B12CF70181917F0155
:1015C000082F10E015950795159507951595079522
:1015D00015950795F80192A18F70650101C0CC0C9B
:1015E0008A95EAF7892F8C2582A30E940F06F801BD
:1015F00022A1C226C2A248855985842795276C81DD
:101600007D812E813F8126273727282339233F8359
:101610002E83FB01E095F095E823F923FD83EC830D
:101620008623972320953095822393234827592793
:1016300059874887882A992A8114910401F1809159
:10164000190290911A0290931402809313028091D0
:1016500023029091240290931E0280931D02809198
:101660002D0290912E029093280280932702809160
:1016700037029091380290933202809331022A9679
:101680006E147F0409F099CFDF91CF911F910F91D4
:10169000FF90EF90DF90CF90BF90AF909F908F9092
:1016A0007F906F9008950E94B4036093B00170938F
:1016B000B1018093B2019093B3010E94C004809164
:1016C0000C02882331F010920C028CE092E00E9410
:1016D000C00A0E943A060C942F0570E090E3899F9F
:1016E000600D711D1124660F771FFB01E950FF4F3C
:1016F0008491FB01E850FF4F94910895EF92FF927F
:101700000F931F93CF93DF93E5EBF1E080E3DF01CD
:101710001D928A95E9F77F0110E01033E1F0C09146
:101720000401D0E0CB51DE4FB1E0C53EDB0771F0E4
:101730000A91E0910201F0910301612F802F099538
:101740008F3F11F49F3F81F3F70100831F5FFFEF8D
:10175000EF1AFF0AE2CFDF91CF911F910F91FF9017
:10176000EF9008950C947E0B90910001891708F07A
:1017700080E091E0909304018093E5010E947E0B4C
:101780000C9408054091040150E090E0682F70E04F
:10179000292F092E000C330B2417350764F42B5125
:1017A0003E4FF9012081022E000C330B261737071C
:1017B00021F09F5FEDCF80E0089581E00895CF9301
:1017C000909100018917A0F4C82F0E94C20B8111CB
:1017D0000FC0E091040181E08E0F80930401F0E0DE
:1017E000EB51FE4FC0830E947E0BCF910C940805F5
:1017F000CF910895CF93DF93D82F0E94C20B8823F7
:1018000081F1C0910401C23028F480E0DF91CF91D2
:101810000C94B40BE5EEF1E090E080E02D2F30E089
:101820004191042E000C550BBC016F5F7F4F421796
:10183000530799F44C2F50E0481B590B6B517E4FC6
:101840008B519E4F0E948B32C150C09304010E9465
:101850007E0BDF91CF910C940805CB016C1700F340
:10186000F6CFDF91CF910895E0910401F0E0EC51C3
:10187000FE4F80818F5F0C94DF0BE0910401F0E05C
:10188000EC51FE4F80810C94FA0BCF93DF93FC0157
:10189000C2819181292F2270C43558F0222309F486
:1018A00050C090FD4EC08CEA8C0FDF91CF910C940C
:1018B000B40BCA32C8F1D6EDDC0FD13251F0D232BE
:1018C00081F4222351F090FD08C0DF91CF910C9458
:1018D000340C2223D1F390FDF8CFDF91CF910C94FB
:1018E0003D0C211110C0A9E4B4E081E38150B9F0AE
:1018F0009C91C91306C011962C91119793812917B9
:1019000001F11296F3CF90FDEECF8D2F0E94C20B06
:10191000811117C08D2FDF91CF910C94DF0B8D2F8C
:10192000DF91CF910C94FA0B222359F090FD09C05E
:101930008C2F0E94C20B882311F08C2FF1CF8C2F9B
:10194000EACFDF91CF910895109209020895CF93C5
:10195000DF9300D000D01F92CDB7DEB7262F342FF3
:10196000842F817041FF15C0811115C080914804FA
:1019700061E0680F609348044FEF5FEF8FEA91E0FA
:101980000F900F900F900F900F90DF91CF910C94CC
:10199000E1098111EBCF0F900F900F900F900F90F6
:1019A000DF91CF9108951F920F920FB60F921124DD
:1019B0008F9381E080930C028F910F900FBE0F9058
:1019C0001F901895FC0182818F5BFB01808381E071
:1019D0000895CF93DF93CDB7DEB769970FB6F8942C
:1019E000DEBF0FBECDBFFC01DB019C919F5F9C93CE
:1019F0009E012D5F3F4F81E1D9011D928A95E9F744
:101A000029E0298384E08A8391E09D8383E08E83AB
:101A10009F8398872A8721E22B879C879D879F87B2
:101A200022E2288B2FE3298B27E02B8B25E02C8BC0
:101A30008E8B20E430E0388F2F8B998F82818B83BF
:101A4000838180688D8B49E150E0BE016F5F7F4FDD
:101A500080E00E94C92C69960FB6F894DEBF0FBED5
:101A6000CDBFDF91CF910895FC01DB018C918138CE
:101A7000A9F413968C911397823281F422811496E3
:101A80008D919C912817190649F48285848F4FE324
:101A900050E061E372E080E80C94C92C90E080E0B3
:101AA0000895FC01DB01228114968D919C9115977C
:101AB0002817190681F511968C9111979C91913AEE
:101AC00069F4813029F0833029F4848D8093F1000A
:101AD00081E008958230F9F4858DF8CF9132D9F400
:101AE0008B3021F412968C91848FF2CF8A3011F4CE
:101AF000158EEECF893079F4CF0116962D913C9159
:101B0000179713964C91423041F461E070E04E9685
:101B10002130310551F080E008954130E1F728305F
:101B20003105C9F768E070E00B960E94EF2CD0CF2A
:101B3000CF93DF93EC0181E08C838D839E01255E42
:101B40003F4F3F832E831986188629E631E039837B
:101B500028836A876C8F8D8F1E8E81EC8B8F0E94FD
:101B60001329BE01DF91CF910C94CF28FC01848D05
:101B70000895EF92FF920F931F93CF93DF938C0101
:101B8000EC012B967C0183E1E80EF11C48E050E06B
:101B9000BE01C7010E947532892B21F1F8018381B2
:101BA00048E050E0BE0180640E94182C8C01E09156
:101BB0006002F0916102309731F09C0148E050E002
:101BC000BE0182E0099588E0FE01D70101900D92E7
:101BD0008A95E1F7C801DF91CF911F910F91FF9096
:101BE000EF9008950FEF1FEFF5CFFC0180E2860F15
:101BF000883070F4605E770B21E030E001C0220F86
:101C00006A95EAF78385822B838781E090E00895C7
:101C1000DF011D9690E080E02D912617B1F3211190
:101C200004C0E80FF91F6587F0CF01968630910553
:101C300099F790E080E00895CF93DF9320E2260F9C
:101C4000283090F4605E770B21E030E001C0220F75
:101C50006A95EAF72095FC0133852323238781E0E9
:101C600090E0DF91CF910895DC011D969C012D5EDF
:101C70003F4FFD014191461303C0EF0121971882A8
:101C8000E217F307B9F720E03D91332349F0EC0167
:101C9000C20FD11D4D853D87ED01219748832F5FF0
:101CA000AE17BF0789F7DBCF0B9628E0FC01119236
:101CB0002A95E9F70895CF93DF93EC010E94540E23
:101CC000CE01DF91CF910C94B90DFC013D96439666
:101CD0002191261729F0E817F907D1F780E0089538
:101CE00081E008952091390230913A0240913B02FF
:101CF00050913C0260913D0270913E0280913F0202
:101D000090914002A1E00E943D322093390230932D
:101D10003A0240933B0250933C0260933D02709321
:101D20003E0280933F02909340020E94493229F480
:101D300061E081E492E00C94980D08958091720224
:101D4000811113C010927B0210927A0280E792E018
:101D500090937D0280937C0289E190E090937F02D2
:101D600080937E0281E0809372020E9486306AE74F
:101D700072E00C94F32FFC0130E020E0419151918E
:101D8000452B41F4220F331F280F391FF9017183AE
:101D9000608308952F5F3F4F2430310579F7089510
:101DA00028E0FC0111922A95E9F70895CF93DF937B
:101DB000EC010E94863028E030E0AE0164E0DF9163
:101DC000CF910C9443300F931F93CF93DF93EC018B
:101DD0008C01085F1F4F48E050E0BC01C8010E9421
:101DE0007532892B51F0CE010E94D60E88E0FE019B
:101DF000D80101900D928A95E1F7DF91CF911F9163
:101E00000F91089528E0FC0111922A95E9F70C94AE
:101E1000E30E0C94020F82E692E00C949E0E8091E9
:101E2000BA02811113C01092C3021092C20289E853
:101E300092E09093C5028093C40281E490E0909375
:101E4000C7028093C60281E08093BA020E94863066
:101E500062EC72E00C94F32FCF93DF93EC010E94BD
:101E60008630AE01435E5F4F2DE130E068E0DF91E8
:101E7000CF910C944330EF92FF920F931F93CF9327
:101E8000DF93EC01F8808D8D8E010F5F1F4F8F1552
:101E9000D9F0F801AE01435E5F4F20E0858D3081BF
:101EA0003196932F9095982319F08323848F21E006
:101EB000E417F50799F7222319F0CE010E942C0FA1
:101EC000FD8ECE010E942C0F7E018EE1E80EF11CEA
:101ED0004CE150E0B801C7010E947532892B81F0B6
:101EE0008CE1F801D70101900D928A95E1F7CE01BE
:101EF000DF91CF911F910F91FF90EF900C942C0FD9
:101F00008FEF9FEFDF91CF911F910F91FF90EF9097
:101F100008956E3D90F4E62FE695E695E695E80F78
:101F2000F92FF11D677021E030E001C0220F6A95A2
:101F3000EAF79181922381E009F480E008956E3DF3
:101F4000A0F4E62FE695E695E695E80FF92FF11D4A
:101F5000677021E030E001C0220F6A95EAF78181C5
:101F6000822B818381E090E00895605E683058F4B0
:101F700041E050E001C0440F6A95EAF7FC0120817E
:101F8000242B2083EFCF90E080E008956E3DA8F4ED
:101F9000E62FE695E695E695E80FF92FF11D6770B7
:101FA00021E030E001C0220F6A95EAF72095818197
:101FB0002823218381E090E00895605E683060F41A
:101FC00021E030E001C0220F6A95EAF72095FC017C
:101FD000308123232083EECF90E080E008952DE12F
:101FE000FC0111922A95E9F70895CF93DF93EC0154
:101FF0000E94EF0FCE01DF91CF910C942C0F80E85F
:1020000092E00C940F0F8091C902811113C01092BD
:10201000D2021092D1028AEC92E09093D402809383
:10202000D30288E190E09093D6028093D50281E0BC
:102030008093C9020E94863061ED72E00C94F32F08
:102040000F931F93CF93DF93EB018A010E94863099
:102050009801AE0165E0DF91CF911F910F910C9433
:102060004330CF93DF931F92CDB7DEB7198241E0A3
:1020700050E0BE016F5F7F4F0E9420100F90DF91F4
:10208000CF9108950C9431100C943110CF93DF93BD
:102090001F92CDB7DEB76983633841F48EE394E0D5
:1020A0000E94022F0F90DF91CF91089541E050E000
:1020B000BE016F5F7F4F0E942010F4CF88EC92E04A
:1020C0000C94031084E690E00C941E044AE050E067
:1020D000682F81EE93E00E941F2A0E94621060E246
:1020E00081EE93E00E945A290C946210FF920F93A4
:1020F0001F93CF93DF93EC01F62E08811981C8015D
:102100000E949D32F81621F06F2DC8010E94A53261
:10211000CE01DF91CF911F910F91FF900895AF9263
:10212000BF92CF92DF92EF92FF920F931F93CF93C4
:10213000DF9300D0CDB7DEB78C016C0184E0C80E10
:10214000D11C5601F12CE12CC7010E949D32F501F2
:1021500081935F01FFEFEF1AFF0A84E0E816F104B4
:1021600099F7F80185818F3FD1F48481982F9F776B
:102170009F3711F487FD148281E0F801858310E018
:1021800000E01A830983F60161916F01CE01019687
:102190000E9476100F5F1F4F0430110591F780E009
:1021A0000F900F90DF91CF911F910F91FF90EF90C3
:1021B000DF90CF90BF90AF9008950F931F93CF9370
:1021C000DF9300D0CDB7DEB77A836983FC0123812A
:1021D00010E000E021110FC000811181CB01800FC0
:1021E000911F9183808342E0BE016F5F7F4F81EE3C
:1021F00092E00E94DA12C8010F900F90DF91CF9108
:102200001F910F910895CF92DF92EF92FF920F935B
:102210001F93CF93DF9300D0CDB7DEB77C016C0165
:1022200084E0C80ED11C10E000E01A830983F60197
:1022300061916F01CE0101960E9476100F5F1F4FD2
:102240000430110591F781E0F70182830F900F9020
:10225000DF91CF911F910F91FF90EF90DF90CF9082
:1022600008951F93CF93DF93EC01162F8091000107
:10227000681748F4862F0E94B40B8C818078912FC8
:102280009F77892B8C831E3720F08C8180788E6716
:102290008C83CE010E9403118C818F77DF91CF91C7
:1022A0001F910895FC01948160FB97F99483892F15
:1022B0008F778F3719F490789E679483CF010C94B1
:1022C0000311CF93DF93EC0181E08B8360E181EE1A
:1022D00092E00E94C1128D81813021F01A82DF913B
:1022E000CF9108952E813F818091E1029091E20289
:1022F0002F3F320769F49F838E83CE010E94031122
:102300008C818F778E3758F7DF91CF910C94B40B77
:102310002817390721F7F4CFFC012381211102C0CE
:102320000E94611180E0089584E090E09093DA02C9
:102330008093D902089581EE93E00E9442279C0188
:1023400081E02A30310529F02F3F3F4F11F080E026
:10235000089508950F931F93CF93DF9300D0CDB7C7
:10236000DEB78B014BE053E08AEE92E00E947E15CF
:10237000811133C06BEF72E0C8010E945E32892B7D
:10238000F1F40E949B1110E000E0811147C00E940F
:102390009B1181113BC041E070E060E081EE93E071
:1023A0000E94942A1A830983CE0101960E94761016
:1023B0000F5F1F4F011584E0180749F727C06FEE24
:1023C00072E0C8010E945E32892B49F062EE72E031
:1023D000C8010E945E32892B69F180E018C08091AB
:1023E000D9029091DA0260E074E0681B790B4AE050
:1023F00050E081EE93E00E94262A0E94621060E283
:1024000081EE93E00E945A290E94621081E00F90B1
:102410000F90DF91CF911F910F910895C8010E94F5
:102420009D320E9466100F5F1F4F011584E0180750
:10243000A9F7ECCF10E000E01A8309836FEFCE011B
:1024400001960E9476100F5F1F4F011584E0180758
:1024500099F787E797E7909301088093000888E150
:102460009BE00FB6F894A895809360000FBE909300
:102470006000FFCFCF93DF93EB0140E653E08AEE9D
:1024800092E00E947E1581117AC049E050E066E535
:1024900073E0CE010E946732892B09F070C0299643
:1024A00069E473E0CE010E945E32892B81F40E94C0
:1024B0009B11811160C041E070E060E081EE93E02B
:1024C0000E94942A89ED92E00E94311140C062E49A
:1024D00073E0CE010E945E32892BE9F16AE373E07A
:1024E000CE010E945E32892B71F166E373E0CE016A
:1024F0000E945E32892B09F042C08091DC02D0E05C
:10250000C0E0882321F0C091DF02D091E002609109
:10251000E1027091E2024AE050E081EE93E00E9415
:10252000262A0E94621064E373E081EE93E00E9429
:1025300036290E9462104AE050E0BE0181EE93E02D
:102540000E94262A15C08091DE020E94661081E05A
:10255000DF91CF9108956091DB028AEE92E00E94B4
:10256000C3150E94621060E281EE93E00E945A2936
:102570000E946210ECCF8091DD028F77E6CF80E081
:10258000E7CFFC01208131812170332781E086175C
:1025900070F4408151815695479551834083220FB5
:1025A000331F41705527242B352B8F5FF0CF31839C
:1025B00020830895DC01FB01415000F181912D91B0
:1025C0003C91119768E070E051E0982F952399F4C1
:1025D000932F991F9927991F220F331F992319F0C1
:1025E00095E029273058550F6150710971F7119600
:1025F0003C932E93E1CF932F9095EBCF089584E6F3
:1026000090E00C941E041F93CF93DF939091E5020A
:10261000891730F080E090E0DF91CF911F9108950D
:10262000C62FD0E090E3899FC00DD11D1124CC0F9F
:10263000DD1F6091E6027091E702C60FD71FCE0141
:102640000E949D32182FCE0101960E949D32912F3B
:10265000E3CF9091E402891710F40C946D0B891B61
:102660000C94031389ED92E00E948F108091000179
:102670008093E40280E0089565EF73E081EE93E0DB
:102680000E9436290E94FF126AE081EE93E00E94C8
:102690005A290E94FF1280E008958093E50290E697
:1026A000899FB001112489ED92E00E94DD10909382
:1026B000E7028093E6020895809300019091DD0285
:1026C00023E033E197FD07C09091E402980F9093C7
:1026D000000129E233E130930301209302010C94BD
:1026E0004D13FF920F931F93CF93DF9300D0CDB77D
:1026F000DEB7F62E672F8C01000F111F8091E602C6
:102700009091E702800F911F9A838983CE010196F1
:102710000E9476108091E6029091E7020196800F68
:10272000911F9A8389836F2DCE0101960E947610A6
:102730000F900F90DF91CF911F910F91FF9008950F
:10274000FF920F931F93CF93DF93F82E8B01C0E07E
:10275000CF15F9F0D0E06D2F8C2FF8010995692F76
:1027600070E0762F6627680F711D4AE050E081EE19
:1027700093E00E94262A0E94FF1260E281EE93E01D
:102780000E945A290E94FF12DF5FD03321F7CF5FEA
:10279000DFCFDF91CF911F910F91FF90089581EED0
:1027A00093E00E9442279C0181E02A30310529F004
:1027B0002F3F3F4F11F080E008950895FF920F934F
:1027C0001F93CF93DF931F92CDB7DEB78B0146ECFB
:1027D00053E08AEE92E00E947E1581118EC047E0A0
:1027E00050E06EEB73E0C8010E946732892B09F05C
:1027F00084C0095F1F4F63EB73E0C8010E945E3223
:10280000892BE1F50E94CF138823B1F06091DD029E
:1028100067FB662760F94AE050E081EE93E00E9492
:102820001F2A0E94FF1260E281EE93E00E945A2963
:102830000E94FF1281E062C041E070E060E081EE42
:1028400093E00E94942A162F698389ED92E00E94FA
:1028500052119091E50290930001112339F083E029
:1028600093E19093030180930201E4CF8091E4020D
:10287000890F8093000189E293E1F3CF6BEA73E063
:10288000C8010E945E32892B39F46DE67BE08091AD
:10289000E4020E94A013CECF64EA73E0C8010E9454
:1028A0005E32892B51F50E94CF1310E000E090E3D7
:1028B000F92E882329F063E073E18091E502E9CFE6
:1028C0000E94CF138111B6CF8091E5028F9DC00188
:1028D00011240817190708F0ADCF41E070E060E05F
:1028E00081EE93E00E94942A272F3327722FC8018C
:1028F0000E9471130F5F1F4FE3CF80E00F90DF91B5
:10290000CF911F910F91FF900895FF920F931F9306
:10291000CF93DF93EC018B01FB01F0800E949D328D
:10292000F81621F06F2DCE010E94A532F801F1803A
:102930002196CE010E949D32F81621F06F2DCE0116
:102940000E94A532C801DF91CF911F910F91FF9096
:102950000895CF92DF92EF92FF920F931F93CF9340
:10296000DF937C0162E070E089ED92E00E94DD106F
:10297000EC01F701918380838C016C01F2E0CF0EB2
:10298000D11C0C151D0540F4C8010E949D328F3FDB
:1029900041F40F5F1F4FF5CF65E071E0CE010E945B
:1029A0008514F701C081D181CE010E949D328093B0
:1029B0000501CE0101960E949D328093060180E0C0
:1029C000DF91CF911F910F91FF90EF90DF90CF900B
:1029D000089566E374E081EE93E00E94362984E670
:1029E00090E00E941E046AE081EE93E00E945A2962
:1029F00084E690E00E941E0480E008950F931F93E8
:102A0000CF93DF93EC018B014CE154E08AEE92E02E
:102A10000E947E15811144C062E074E0C8010E94EA
:102A20005E32892BE9F581EE93E00E9442278A30DD
:102A30009105C9F00196B9F041E070E060E081EEE7
:102A400093E00E94942A609305017093060165E06B
:102A500071E0888199810E94851481E0DF91CF9196
:102A60001F910F9108956091060170E0762F6627FF
:102A700080910501680F711D4AE050E081EE93E0FE
:102A80000E94262A84E690E00E941E0460E281EE05
:102A900093E00E945A2984E690E00E941E04D7CF5A
:102AA00080E0DCCFCF93DF93DC01EB019A818C9146
:102AB000981305C02B8111968C91281749F09E37E9
:102AC00021F080E0DF91CF9108958B81813DC9F79E
:102AD000898181FFF6CF80FDF4CF87FDF2CF82E1BF
:102AE00091E00E94E21B882361F361E082E191E0C2
:102AF0000E94461C1A821B8281E0E4CFCF93DF93B1
:102B0000CB01EA016EE774E00E945E32892B49F442
:102B1000BE0181EE93E00E94652981E0DF91CF91B3
:102B2000089580E0FBCFCF93DF93EB0144E654E0C0
:102B30000E947E15811125C067E574E0CE010E94D8
:102B40005E32892B89F487E797E790930108809399
:102B5000000888E19BE00FB6F894A8958093600088
:102B60000FBE90936000FFCF6FE474E0CE010E942F
:102B70005E32892B31F40E948A0481E0DF91CF918B
:102B8000089580E0FBCF611106C064E474E081EE3B
:102B900093E00C9436296AE474E0F9CF10920A03AA
:102BA0000895CF93DF93EC0181EE93E00E945827C4
:102BB00081EE93E00E945B27892B09F45BC081EED4
:102BC00093E00E946B27E8A191E09E0F98A3EC0F81
:102BD000FD2FF11D8083FE01E90FF11D31978081EA
:102BE000803271F0903260F481EE93E00E945B27B6
:102BF000892B31F081EE93E00E9442270A97F9F683
:102C00008881811107C018A280E2FE0111928A9585
:102C1000E9F730C0E8A1EC0FFD2FF11D319780815D
:102C20008032F9F4E8A1E150FF0BEC0FFD1F808129
:102C3000803209F41082CE010E94EF0581EE93E00C
:102C40000E945B27892B31F081EE93E00E946B2775
:102C50008A30A1F763E874E081EE93E00E94652971
:102C6000D2CF81EE93E00E9442270A97D9F288A141
:102C70008032C0F680E0DF91CF910895FC0184910D
:102C80003196949108958F929F92AF92BF92FF9246
:102C90000F931F93CF93DF93EB01209709F4A4C008
:102CA000F12C8E010F5F1F4FFE018491EFEFE80FB3
:102CB000ED3008F099C0F0E0E05AF94E0C941D3266
:102CC0009D16A916B216BF16CC16D916E216EB162B
:102CD000A116A116A1166D1688168F2C912CB12C59
:102CE000A12CB801F80184916F5F7F4F0E5F1F4FD9
:102CF000FB016491611102C0882319F1782F8CE0E7
:102D000093E00E945518C501B4010E94E503E9CF84
:102D10008F2C912CB12CA12C0F5F1F4FF8013197F4
:102D20006491662371F070E08CE093E00E94551886
:102D3000C501B4010E94E503EFCF2296F801F4909B
:102D40008E016F2D70E090E080E00E94E503E801C5
:102D5000A8CF2296F801649170E090E080E00E9494
:102D6000E503EECFF80174918E010D5F1F4FFE0158
:102D7000329664918CE093E00E94B117E2CFF801A3
:102D800074918E010D5F1F4FFE01329664918CE0AD
:102D900093E00E94EC17D5CFF80174918E010D5F7E
:102DA0001F4FFE01329664918CE093E00E9455180B
:102DB000C8CF2296F801649170E08CE093E00E9405
:102DC000B117BECF2296F801649170E08CE093E0D9
:102DD0000E94EC17B5CF2296F801649170E08CE068
:102DE00093E00E945518ACCFDF91CF911F910F91C6
:102DF000FF90BF90AF909F908F900895862F90E0A6
:102E00006134E0F46A33B0F5603269F170F46A302D
:102E100039F130F482E2683050F590E080E00895B6
:102E20006B31D9F790E089E208956133F8F4880FA7
:102E3000991F845B9B4F0E943E160895613638F4BB
:102E40006B35E8F0880F991F8A5F9B4FF4CF6B3783
:102E5000D0F06F3710F7880F991F8E529C4FEBCF31
:102E600090E088E2089590E08CE208958DEE860F60
:102E700090E00895880F991F865C9B4FDCCF83EC10
:102E8000860F98E0089583EAF2CF0F931F93CF93B4
:102E9000DF938C01EB01FE016491662371F0C801A0
:102EA0000E94FE16811102C0992329F0BC018CE01A
:102EB00093E00E9455182196EECF90E080E0DF91DC
:102EC000CF911F910F9108950F931F93CF93DF938D
:102ED000EB012B8130E0322F22274A8150E0BA01EA
:102EE0007056260F371F2F3F310509F0F8F48C017B
:102EF000BE01842F0E944505BC01C8010E944316F3
:102F0000898180FF02C081FF0DC08A8190E09056C8
:102F10002B8130E0322F2227820F931F8F3F9105A4
:102F200029F020F08CE093E00E94141880E0DF91FB
:102F3000CF911F910F91089567E874E081EE93E0BF
:102F40000E94362984E690E00E941E046AE081EE29
:102F500093E00E945A2984E690E00E941E0480E0DB
:102F60000895EF92FF920F931F93CF93DF9300D0BA
:102F700000D01F92CDB7DEB78C01F62EE72E609100
:102F800048048FEF898382E88A83FB827C836D8388
:102F90002FEF32E84F2D572F8FEA91E00E942D0935
:102FA000C8014096F801E817F90741F02081211186
:102FB00011C0218121110EC0F082E1820F900F908B
:102FC0000F900F900F90DF91CF911F910F91FF9075
:102FD000EF9008953296E7CFCF93DF9300D000D0E3
:102FE0001F92CDB7DEB7AB019C01205F3F4FFC01C4
:102FF0002E173F0751F08081841305C0818185130E
:1030000002C0108211823296F3CF609148042FEFF4
:1030100031E88FEA91E00F900F900F900F900F9092
:10302000DF91CF910C942D09CF92DF92EF92FF9216
:103030000F931F93CF93DF9300D000D01F92CDB793
:10304000DEB77C0120E1E20EF11C8C01DD24DA9474
:1030500081E8C82EE016F106D1F0F80140815181D7
:10306000411102C0552381F060914804D982CA827F
:103070004B835C836D832FEF31E88FEA91E00E94F0
:103080002D09F801108211820E5F1F4FE3CF0F90C0
:103090000F900F900F900F90DF91CF911F910F9194
:1030A000FF90EF90DF90CF9008950F931F93CF93F1
:1030B000DF9300D000D01F92CDB7DEB78B016091B7
:1030C00048042FEF32E8A8018FEA91E00E942D0911
:1030D000609148042FEF31E8A8018FEA91E00F904A
:1030E0000F900F900F900F90DF91CF911F910F9144
:1030F0000C942D090F931F93CF93DF938C01005FE6
:103100001F4FEC010C171D0771F0688179818981CF
:103110009881911102C0882321F08FEA91E00E94EA
:1031200017082296EFCF80E0DF91CF911F910F918A
:10313000089560ED74E081EE93E00E94362984E604
:1031400090E00E941E046AE081EE93E00E945A29FA
:1031500084E690E00E941E0480E00895CF93DF9300
:1031600000D000D000D0CDB7DEB786EC94E00E944E
:10317000F830EAEDF4E0108A868597852485358558
:1031800019823B832A839D838C831E820284F3856C
:10319000E02D0190F081E02D46E050E0BE016F5F30
:1031A0007F4F84EE94E0099580E026960FB6F89460
:1031B000DEBF0FBECDBFDF91CF910895FC0170350A
:1031C00079F4862F8076803429F49085862F8F7B42
:1031D000892B8087862F807729F48781682B6783E6
:1031E00080E008958031E1F780E1689FB00111240B
:1031F000F4CFCF93DF93EC0186EC94E00E94BB30D8
:10320000688586EC94E00E94C13086EC94E0DF9102
:10321000CF910C94D330FB01928196FB222720F9A9
:1032200080E090FD82E0822B20E091FD24E0822B63
:1032300020E092FD28E0822B93FD04C090E0892BD2
:103240000C94561A90E1FBCFFB012381203559F4F1
:10325000DC0117961C9217972281322F307630347A
:1032600021F418961C9280E0089525FFFCCF21815F
:1032700021FFF9CF20FDF7CF0E940B19F4CF209149
:10328000B0013091B101FC01318320839681892FF7
:103290008F7019F410922703089580910F01819582
:1032A00092FF80E093FF03C020910F01820F609195
:1032B0000F01619590FF60E091FF03C090910F01B5
:1032C000690F0E94F81A86EC94E00C94D3300F93A7
:1032D0002091B0013091B101FC01358324838681B6
:1032E00090E024E0959587952A95E1F70097F1F015
:1032F00000910901019582FF00E083FF03C0209146
:103300000901020F2091090180FF20E081FF03C025
:1033100080910901281B40E060E086EC94E00E9467
:10332000B33086EC94E00F910C94D3300F91089554
:10333000CF93DF93EC018091B0019091B1012A818C
:103340003B81AC01421B530B9A0140910A01509101
:103350000B012417350780F09B838A832091270374
:1033600030910C014FEF50E0431B51092417150613
:103370001CF4230F2093270328813981821B930B90
:1033800020910D0130910E018217930718F0CE01A4
:103390000E943F198091B0019091B1012C813D8133
:1033A000821B930B2091070130910801821793072C
:1033B00018F0CE010E94671980E0DF91CF91089547
:1033C0000F931F93CF93DF93FB0123812035C9F423
:1033D0008B01EC0182818076803419F4CE010E9449
:1033E000F9188F818E831F82F8018281807779F4AA
:1033F0008091B0019091B1019B838A83CE010E949C
:103400003F1980E0DF91CF911F910F910895803196
:10341000C1F7CE010E946719F4CFCF93DF9300D09C
:1034200000D000D0CDB7DEB736952795820F931F19
:1034300056954795640F751FEAEDF4E095878487EC
:1034400077876687208929839B838A837D836C8322
:103450001E820284F385E02D0190F081E02D46E08C
:1034600050E0BE016F5F7F4F84EE94E00995269691
:103470000FB6F894DEBF0FBECDBFDF91CF91089598
:1034800010922A031092290310922C0310922B03FE
:103490008FEF9FE79093300380932F0390932E0339
:1034A00080932D0381E08093280308950F931F9349
:1034B000CF93C82F80912803811102C00E94401A27
:1034C000C0FF06C010922803CF911F910F9108955D
:1034D000E09111010E2F10E080912F0390913003A5
:1034E000B8010E94D3319B017093300360932F0386
:1034F00080912D0390912E03B8010E94D331AB012E
:1035000070932E0360932D036C2F6470E0912B0356
:10351000F0912C038091290390912A037C2F7670DF
:10352000763091F4820F931F90932A03809329039E
:10353000BA016E0F7F1F70932C0360932B03CF9102
:103540001F910F910C940D1A662349F1D801119720
:10355000A49FB001A59F700DB49F700D1124E60FBC
:10356000F71FF0932C03E0932B03C4FF1DC0015001
:103570001109029FB001039F700D129F700D11245D
:10358000860F971F90932A038093290360912B0342
:1035900070912C038091290390912A03D0CFC1FD13
:1035A000E4CFE40FF51FDDCFC3FDF0CF820F931FF3
:1035B000E9CF482F50E087FD0AC0889FC001112441
:1035C000880F892F881F990B91958F5F089520E0B0
:1035D00031E0241B350B229FC001239F900D900DDD
:1035E0001124880F892F881F990B91958095089534
:1035F000EF92FF920F931F93CF93DF93082F162F15
:10360000C0911001D0E0F12CE12C8823D1F0809101
:1036100027030E94D91A20912603382F0303C001E3
:103620001124820F911D27FD9A957E01C817D90795
:1036300044F0EE24FF24EC1AFD0AE816F9060CF417
:103640007C01112309F449C0809127030E94D91AF3
:1036500020912503382F1303C0011124820F911DDF
:1036600027FD9A95C817D9073CF0D195C195D10986
:10367000C817D9070CF4EC0110922803AE01D7FF4C
:1036800002C0415F5F4F94E0559547959A95E1F7E9
:10369000B701F7FE02C0615F7F4F84E075956795C3
:1036A0008A95E1F700E020E086EC94E00E94B330D8
:1036B00020E130E0C701B9010E94E7318093260381
:1036C000CE01B9010E94E73180932503DF91CF91AC
:1036D0001F910F91FF90EF900895D0E0C0E0CCCF04
:1036E000FC018281DB019C91891730F5A081B181B9
:1036F000A80FB11D2C9130E0938102C0359527951C
:103700009A95E2F724834481442391F0242F30E0FA
:10371000938140FF07C0880F880F880F890F85832A
:1037200081E008953595279524839F5F9383EBCFA0
:103730008F5F82831382D5CF80E00895262F269550
:1037400026952695820F911DFC01808190E067707F
:1037500002C0959587956A95E2F781700895E62FE6
:10376000E695E695E695E80FF92FF11D677081E083
:1037700090E0A0E0B0E004C0880F991FAA1FBB1F13
:103780006A95D2F72081822B80830895E62FE695F3
:10379000E695E695E80FF92FF11D862F877041E039
:1037A00050E060E070E004C0440F551F661F771FB3
:1037B0008A95D2F740955095609570958081482301
:1037C00040830895EF92FF920F931F93CF93DF935F
:1037D000CDB7DEB72C970FB6F894DEBF0FBECDBFC6
:1037E0008C010A9698878F8319861A86FF24FA948B
:1037F000FC869A83898386E0E82EEB821C82FE8217
:10380000BE016D5F7F4FCE0107960E94701B811134
:1038100013C0005F1F4F18870F8319861A86FC8616
:103820001A830983EB821C82FE82BE016D5F7F4F8B
:10383000CE0107960E94701B2C960FB6F894DEBF3F
:103840000FBECDBFDF91CF911F910F91FF90EF90F1
:103850000895272F207C69F4605E683098F4FC019D
:103860008681978102C0969587956A95E2F7817067
:103870000895743439F426ED260F2A3218F4625272
:10388000603168F381E008950C94291CAF92BF92D7
:10389000DF92EF92FF920F931F93CF93DF93CDB7F9
:1038A000DEB761970FB6F894DEBF0FBECDBF8C01B7
:1038B0000A967C01662381F1580190E1A90EB11CA2
:1038C000B886AF8219861A868FEF8C87BA82A98252
:1038D00096E09B831C828E83BE016D5F7F4FCE017D
:1038E00007960E94701B8823B9F0DC846D2DC501FA
:1038F0000E94C61B6D2DC7010E94C61B6091480423
:103900002D2D31E84FEF5FEF8FEA91E00E942D09F6
:103910008A858F5F8A87E0CFF886EF8219861A86BC
:103920008FEF8C87FA82E98296E09B831C828E83DC
:10393000005F1F4FBE016D5F7F4FCE0107960E9453
:10394000701B882309F1DC846D2DC8010E949E1B29
:103950006D2D8823A9F0C8010E94C61B6D2DC701DB
:103960000E94C61B609148042D2D31E84FEF5FEF98
:103970008FEA91E00E942D098A858F5F8A87DACFCE
:10398000C7010E94C61BF8CF61960FB6F894DEBF40
:103990000FBECDBFDF91CF911F910F91FF90EF90A0
:1039A000DF90BF90AF9008956AED74E081EE93E0F0
:1039B0000E94362984E690E00E941E046AE081EEAF
:1039C00093E00E945A2984E690E00E941E0480E061
:1039D00008954F925F926F927F928F929F92AF92D3
:1039E000BF92CF92DF92EF92FF920F931F93CF93EC
:1039F000DF93CDB7DEB761970FB6F894DEBF0FBE89
:103A0000CDBF8C01FC0160807180C090B001D0906E
:103A1000B10186899789C81AD90A82809380780172
:103A2000FAE0EF0EF11CF886EF8219861A868FEF06
:103A30008C87FA82E98296E09B831C828E83512CCC
:103A4000580180E1A80EB11CBE016D5F7F4FCE0111
:103A500007960E94701B482E882349F15C84652DCF
:103A6000C5010E949E1B8823D1F0C614D70490F094
:103A7000652DC5010E94C61B652DC7010E94C61B8E
:103A800060914804252D31E84FEF5FEF8FEA91E018
:103A90000E942D098A858F5F8A87542CD5CFC81440
:103AA000D904C0F3652DC7010E94C61BF3CF511086
:103AB00007C08091B0019091B101F801978B868B7E
:103AC00080E061960FB6F894DEBF0FBECDBFDF91E8
:103AD000CF911F910F91FF90EF90DF90CF90BF900B
:103AE000AF909F908F907F906F905F904F900895D0
:103AF0000C94E91C872F90E0982F8827860F911D42
:103B00002FEF280F283018F4815290E008958F5D30
:103B100094E40895AF92BF92CF92DF92EF92FF921A
:103B20000F931F93CF93DF93FB01B180B7FC5BC072
:103B3000EB018C016C01FAE0CF0ED11C6881C6014B
:103B40000E949E1BA82E780180E1E80EF11C68817E
:103B5000C7010E949E1BB1FE90C0B0FC8EC0A11098
:103B600051C0811185C08A819B81292F30E0322F7D
:103B70002227482F50E04150504C240F351F203150
:103B8000310598F46A817B81C8010E947A1D9B836C
:103B90008A836881C6010E94AF1B8091B001909119
:103BA000B101F801978B868B1BC0F8012085222379
:103BB00039F0292F207C21F420E2280F283048F307
:103BC000F8012185222331F0943421F426ED280FC9
:103BD0002A32F8F2292F207C41F4805E883050F49C
:103BE0008881F801808F80E038C0943419F48A52BB
:103BF0008A32B0F3F8018689978920813181821B4E
:103C0000930BD0CF882361F36881C6010E94C61B45
:103C10009881F801808D981729F06881C7010E946A
:103C2000C61BDECF6A817B81C8010E94441C8823A9
:103C3000A1F3F8018481958197FF02C08081918171
:103C40002091B0013091B101F80146895789241BB8
:103C5000350B2817390708F782E0DF91CF911F91C4
:103C60000F91FF90EF90DF90CF90BF90AF900895AD
:103C70006881C6010E94C61BD0CFA11003C0882353
:103C800009F4B1CF6881C7010E94AF1BE5CF62EE96
:103C900074E081EE93E00E94362984E690E00E9471
:103CA0001E046AE081EE93E00E945A2984E690E0C7
:103CB0000E941E0480E00895FC01872F90E0982F59
:103CC0008827680F792F711D613180EC7807E0F04B
:103CD000623188EC780750F46151704C66A717A6E2
:103CE00011AA80EE870F80AB81E00895633180EDEB
:103CF000780750F46251784C66A717A68AE2870FBE
:103D000080AB84E481ABF0CF80E008958F929F92E6
:103D1000AF92BF92CF92DF92EF92FF920F931F93D9
:103D2000CF93DF9300D000D0CDB7DEB78C01F62E55
:103D30002FE2261708F469C0E62FF0E0EE0FFF1F10
:103D4000E75BFB4FD080E1808FEFD8120FC0E81205
:103D50000DC0AF2DB0E0AB54BE4FE0910201F09129
:103D600003016F2D8C910995D82EE92E6D2D7E2D96
:103D7000C8010E945C1EB82E811135C0EF2DF0E005
:103D8000EB54FE4F8080C12CAA24AA94912CF801F8
:103D90008281C81608F042C0F4E0CF9EC001112411
:103DA000F80160817181680F791FAA8244E050E0B8
:103DB000CE0101960E94553289819A813B812C81E6
:103DC000F9122AC0482F082E000C550B481559052A
:103DD00011F08F3F09F5F801D6A6E7A6C90190AB0F
:103DE00021ABBB24B3948B2D0F900F900F900F90AD
:103DF000DF91CF911F910F91FF90EF90DF90CF90C7
:103E0000BF90AF909F908F9008951092A904109248
:103E1000AA04E9EAF4E096CFC394B9CFD6A6E7A600
:103E20008FEF80AB81ABDFCFCF93DF93FC01EB0152
:103E30009A01261B370BA4E6B0E00E94233226A18C
:103E400030E050E040E00E94FB318091B001909161
:103E5000B101BC016C1B7D0B81E06217730708F098
:103E600080E0DF91CF910895292F207C39F490E2F2
:103E7000980F81E0983048F080E007C09434E1F773
:103E800096ED980F81E09A32B8F70895CF93DF93BB
:103E9000EC018881681780F5882371F1815088834F
:103EA000E62FF0E0DF011196AC0FBD1FEE0FFF1FF4
:103EB0007196EC0FFD1F962F981780F411962C9198
:103EC00011972D9318962C91189717962C93179756
:103ED00022813381219331939F5FEECF2FEF30E02A
:103EE00001C0220F6A95EAF789A1922F9095982335
:103EF00086958223892B89A3DF91CF910895CF9353
:103F0000DF9300D000D01F92CDB7DEB7FC0134851F
:103F100084A1982F917080FD28C082E0248139838C
:103F20008A836B837C832D8391110AC0872F90E055
:103F3000982F8827680F792F711D64307105F0F470
:103F400060E0CF0103960E94461F29813A814B8190
:103F50005C816D818FEA91E00F900F900F900F9030
:103F60000F90DF91CF910C94E10981E0D7CF6D32B2
:103F7000710530F36933710518F703C068327105B4
:103F8000B0F78489958994A783A7DACFCF93DF937D
:103F9000FC017381DC011D9681E090E060E08717F1
:103FA000F0F452A94D9124A130E0082E02C03595BD
:103FB00027950A94E2F720FD0DC0541721F080E008
:103FC000DF91CF9108952489358934AB23AB682FD5
:103FD0000196E5CF5413FCCF8FEF82ABF0CF8091E9
:103FE000B0019091B10123A934A9821B930B25A99B
:103FF0002817190609F068F48FEF82AB6623F9F2EF
:10400000EF012396CE010E94461F60E0CE010E9480
:10401000461F81E0D5CF7F928F929F92AF92BF9241
:10402000CF92DF92EF92FF920F931F93CF93DF9384
:10403000EC019B81911110C0F12C8F2DDF91CF915C
:104040001F910F91FF90EF90DF90CF90BF90AF90B6
:104050009F908F907F9008959C848CA180FF13C0C7
:10406000983041F460E070E0CE010E947F1FFF2491
:10407000F394E3CF8AA99812F5CFCE010E94C61F10
:104080008111DACFEFCF692DCE010E94861E8823E1
:1040900009F470C0FDA0FF2009F46CC00EA51FA597
:1040A000C8010E94341F882E8091B0019091B10107
:1040B0002BA53CA5821B930B2AA52817190609F0EE
:1040C00010F57B80A090B001B090B1016E0101E0CD
:1040D00010E0E12C202F071508F065C08CA190E0BE
:1040E000002E02C0959587950A94E2F780FD12C0D4
:1040F000811040C0EE2009F454C07FEFC71AD70AE0
:104100000F5F1F4FE7CF8110DCCFB801CE010E94B7
:104110007F1FD7CFF6019585FE013D9681E099126C
:104120002DC0EE2019F08EA1811110C0882059F009
:1041300068A979A99AAA8C899D899CAB8BABCE0181
:104140000E947F1F7ACF6EA57FA5F4CFF801EE0FF6
:10415000FF1FEC0FFD1F44895589EE2DF0E0EE0F97
:10416000FF1FEC0FFD1F64897589CE010E94141F8B
:104170008111C3CF6EA57FA577CF8F5F821708F01F
:10418000BCCF31913913F9CF4C895D89B501641BDE
:10419000750B39A53617170609F078F768A979A9BC
:1041A000CECFE02EAACF88E0781246CFE3CF0F9390
:1041B0001F93CF93DF93EC01FB0124818DA5922FF8
:1041C000981B19162CF08B8181111CC080E025C032
:1041D0002DA780818033D0F7818187FDF7CF8B01B8
:1041E0008DA181111FC062817381CE010E945C1E6E
:1041F000882361F38EA59FA5D80113969C938E9377
:104200001297E4CF022E000C330B8C81281B31094E
:1042100087FD339537FDDACF82E0DF91CF911F9193
:104220000F9108952B81822F90E03481FE01E80FD9
:10423000F91F3483DB013C913487880F991FFE01FD
:10424000E80FF91F8091B0019091B101958B848B9B
:1042500011964C913CA181E090E0A0E0B0E0022EEC
:1042600004C0880F991FAA1FBB1F0A94D2F740FFF2
:104270000CC041FD0AC0832B8CA32F5F2B83CE0182
:104280000E940B208111FBCFC7CF80958323F4CFF1
:104290000F931F93CF93DF93EC012091B0013091E6
:1042A000B1018AA590E04BA55CA5B901641B750B13
:1042B0006817790738F0A90141505109481B590B7B
:1042C0005CA74BA78B818823D9F08C899D89281BFB
:1042D000390B8FA198A52817390768F00EA51FA5DF
:1042E000C8010E94341FB801811102C068A979A9D0
:1042F000CE010E947F1FCE010E940B208111FBCFB7
:1043000080E0DF91CF911F910F910895CF93DF93BC
:10431000C1E3D3E0198218821A821B8288E0E0E4AC
:10432000F1E0ADE3B3E001900D928A95E1F781E011
:104330008DA380E58EA38AEF90E098A78FA382E3F8
:1043400089A78BE48AA780E091E09CA78BA78FEFD9
:104350008DA78EA78FA788AB89AB8AAB88EC8DAB76
:10436000DF91CF910895FC018FEF818312824091FC
:1043700048015091490160914A0170914B01478376
:10438000508761877287848B80917C0381112CC058
:1043900081EE809384031092850386E280938603E6
:1043A00088E080938703109289031092880395EE2A
:1043B00090938A0310928B0397E290938C038093DF
:1043C0008D0310928F0310928E031092900310921F
:1043D00091031092920310929303109295031092FE
:1043E000940381E080937C0384E893E090939703A7
:1043F00080939603089569EE74E081EE93E00E9445
:10440000362984E690E00E941E046AE081EE93E083
:104410000E945A2984E690E00E941E0480E00895DC
:1044200080E026E0E0919603F0919703829FE00DF3
:10443000F11D1124908191110FC0318131110CC0F7
:104440003281311109C03381311106C04481558157
:10445000452B11F48FEF0895961303C091819717A0
:1044600011F08F5FDFCF08950F931F93CF93DF93EA
:10447000CDB7DEB72A970FB6F894DEBF0FBECDBF1B
:104480008C01FC01838980FD48C082E0F80127810E
:1044900093812E838F838FEF888789879A876623FE
:1044A00021F1948997FD21C09081923079F4609137
:1044B0004804298391E09A838B838C836D8331E058
:1044C0004FEF5FEF8FEA91E00E942D09F801848998
:1044D000E0919603F091970396E08902E00DF11DBB
:1044E00011248281938199878887F80182818823AA
:1044F000E1F0815082833396D8011B9690E09817A3
:1045000070F4218121932481238312962D913C9173
:1045100013972D933D939F5FF2CF81E0B7CFF801C2
:10452000838990E095958795838B2E813F8148857F
:1045300059856A858FEA91E02A960FB6F894DEBF16
:104540000FBECDBFDF91CF911F910F910C94E10968
:10455000CF93DF93EC018A81882329F060E0CE01BC
:104560000E943422F8CFDF91CF910895FC0182811F
:10457000882311F120912B0130912C018489A09185
:104580009603B091970396E08902A00DB11D112406
:1045900014968D919C91009709F09C018091B00137
:1045A0009091B10143855485841B950B8217930725
:1045B00018F0CF010E94A82280E00895CF93DF93E6
:1045C000FC01EB012081822F90E03C81DF01A80FEC
:1045D000B91F11963C931197388115963C93880F1B
:1045E000991FDF01A80FB91F8091B0019091B1010F
:1045F0001A969C938E9319979981818941E050E096
:1046000060E070E0022E04C0440F551F661F771F44
:104610000A94D2F790FF09C091FD07C0482B418B47
:104620002F5F2083DF91CF91089540954823F7CFE6
:104630000F931F93CF93DF93EC01FB01848199814A
:10464000282F291B12164CF09A8191111CC080E072
:10465000DF91CF911F910F9108958983208120339D
:10466000B0F7818187FDF3CF382F327081FF1FC0F3
:1046700080FD1DC09281983591F49381913DB9F4EC
:10468000188281E0E5CF082E000C990B2B81821B4C
:10469000910927FD939597FDDACF82E0D9CF99351F
:1046A00031F49381913D19F481E08883D1CF9881D1
:1046B000913069F28F019A81992371F080FF09C0CE
:1046C000311107C08F81821323C061E0CE010E94A7
:1046D0003422CE010E94A822F801818181FFB7CF48
:1046E00080FDB5CF62817381CE010E9410228C8B38
:1046F00087FDADCF8881823069F4F8012081318156
:104700004281538164818FEA91E00E942D0902C0A9
:104710009430F9F2B801CE0102960E94DE22BDCF9C
:1047200087E693E00C94B3210C949D328F929F9274
:10473000AF92BF92CF92DF92EF92FF920F931F93AF
:10474000CF93DF938C01FC01E080F180158214820D
:10475000C280D380CE0CDF1C4701B12C8C149D0489
:1047600008F04BC0E4012196C4010E9494238E30CE
:1047700008F043C0E82FF0E0E054FC4D0C941D32EB
:10478000EF23CE23CE23D223D223D223CE23CE2374
:10479000CE23D023D023D023D523E423E4012296B3
:1047A0004E01DCCFE4012396FBCF4E01CE010E94E7
:1047B0009423A82E2296C40101960E949423A1104E
:1047C000F4CF8111F2CFECCF2C2F9D2F2196822F89
:1047D0000E9494232C2F9D2F8111F8CFE1CFB39409
:1047E000EB2DF0E03296EE0FFF1FE00FF11FCE0130
:1047F0008E199F0991838083D3CF8B2DDF91CF9129
:104800001F910F91FF90EF90DF90CF90BF90AF90EE
:104810009F908F9008958F929F92AF92BF92CF9268
:10482000DF92EF92FF920F931F93CF93DF93FC01E0
:10483000EC5BFF4F2081621708F0DFC07C01E62FA0
:10484000F0E03296EE0FFF1FEE0DFF1DD7010D9128
:104850001C9180819181080F191FD12CF701808153
:10486000918122813381820F931F0817190708F065
:10487000C4C0E8012196C8010E94942381508D3064
:1048800008F0BBC0E82FF0E0E85BFB4D0C941D3254
:10489000742483248F24A024B124C224CE24DA24B7
:1048A0007B247B247B245524E6248D2C912CB12C55
:1048B000A12CCE010E949423C82E8E010E5F1F4FA3
:1048C000CE0101960E949423811102C0CC2091F068
:1048D000682F7C2D8CE093E00E945518C501B4012F
:1048E0000E94E503E801E5CF0E5F1F4FCE010E9455
:1048F0009423D82EE8016D2D70E090E080E00E94B6
:10490000E5038E01ABCF0E5F1F4FCE010E949423B3
:10491000682F70E090E080E00E94E503EBCFCE01CD
:104920000E949423C82EE8012396C80102960E9493
:104930009423682F7C2D8CE093E00E94B117DBCF8D
:10494000CE010E949423C82EE8012396C801029646
:104950000E949423682F7C2D8CE093E00E94EC173A
:10496000CACFCE010E949423C82EE8012396C80125
:1049700002960E949423682F7C2D8CE093E00E9485
:104980005518B9CF0E5F1F4FCE010E949423682F98
:1049900070E08CE093E00E94B117ACCF0E5F1F4F28
:1049A000CE010E949423682F70E08CE093E00E9477
:1049B000EC17A0CF0E5F1F4FCE010E949423682FEB
:1049C00070E08CE093E00E94551894CFCE018D2CBE
:1049D000912CB12CA12C21960E949423882309F4B8
:1049E0008ACF682F70E08CE093E00E945518C501D3
:1049F000B4010E94E503CE01EECFDF91CF911F916C
:104A00000F91FF90EF90DF90CF90BF90AF909F906D
:104A10008F900895292F30E0322F222790E08C5577
:104A2000914D280F391F81E02032310508F080E0D8
:104A300008950F931F93CF93DF938C01EB018A812D
:104A40009B810E940A258823A9F0898181FF0DC0DE
:104A500080FD0BC06A816C55C8010E940B2481E067
:104A6000DF91CF911F910F9108958CE093E00E9408
:104A70001418F5CF80E0F4CF62E275E081EE93E0A8
:104A80000E94362984E690E00E941E046AE081EECE
:104A900093E00E945A2984E690E00E941E0480E080
:104AA00008950F931F93CF93DF93EC018B0189ED52
:104AB00092E00E94DD10998388831B830A83CE01D4
:104AC0000E949623CC5BDF4F8883DF91CF911F91AB
:104AD0000F910895BF92CF92DF92EF92FF920F93C2
:104AE0001F93CF93DF93EC018B0148E055E08AEEF2
:104AF00092E00E947E15811186C047E050E060E0A0
:104B000075E0C8010E946732892B09F07CC0095FFB
:104B10001F4F6CEF74E0C8010E945E32892B09F0D0
:104B20005FC081EE93E00E944227F12CE12C8A3095
:104B3000910511F0019621F58A819B81E816F9060D
:104B400008F04EC0888199818E0D9F1D0E9494238C
:104B50004AE050E0682F81EE93E00E941F2A84E62D
:104B600090E00E941E0460E281EE93E00E945A29C8
:104B700084E690E00E941E048FEFE81AF80ADCCF6A
:104B800081EE93E00E9442278A30910511F101964F
:104B900001F18A819B81E816F906D8F441E070E0C2
:104BA00060E081EE93E00E94942AB62E67018FEFB9
:104BB000C81AD80A88819981E80EF91EC7010E9497
:104BC0009D32B81621F06B2DC7010E94A5327601E7
:104BD000D7CFCE010E949623FE01EC5BFF4F80836E
:104BE00064EF74E0C8010E945E32892B51F441E009
:104BF00070E060E081EE93E00E94942ACE010E9472
:104C00000B2481E001C080E0DF91CF911F910F91D3
:104C1000FF90EF90DF90CF90BF90089584E690E0F2
:104C20000C941E046AE575E081EE93E00E9436293B
:104C30000E940E266AE081EE93E00E945A290E94AB
:104C40000E2680E008950F931F93CF93DF93EC011E
:104C50008B0189ED92E00E94DD10998388831B838C
:104C60000A83DF91CF911F910F9108957F928F92C8
:104C70009F92AF92BF92CF92DF92EF92FF920F93EB
:104C80001F93CF93DF9300D0CDB7DEB77C018B01AC
:104C900048E455E08AEE92E00E947E158111DAC068
:104CA00066E375E0C8010E945E32892B09F0D2C02C
:104CB00081EE93E00E94422710E000E08A309105E7
:104CC00019F0019609F080C0F701828093800815E1
:104CD000190508F046C05801FFEFAF1ABF0AF701E7
:104CE00080819181800F911F0E949D32C82E8FEF8D
:104CF0008C0D8E3FB0F54AE050E06C2D81EE93E0D4
:104D00000E941F2A0E940E2660E281EE93E00E941C
:104D10005A290E940E26D12C4501FFEF8F1A9F0AB7
:104D2000F701808191818A0D9B1D0E949D32682F21
:104D300081EE93E00E945A290E940E2681E08D0D9B
:104D400054018C110CC00E5F1F4F0D0D111D6AE038
:104D500081EE93E00E945A290E940E26B5CFD82EEC
:104D6000DBCF4AE050E070E060E081EE93E00E942B
:104D70000B2A0E940E2660E281EE93E00E945A29DF
:104D80000E940E2660E375E081EE93E00E943629D2
:104D90000E940E264AE050E0B40181EE93E00E94AA
:104DA000262A0E940E2681E00F900F90DF91CF916E
:104DB0001F910F91FF90EF90DF90CF90BF90AF9039
:104DC0009F908F907F900895F701828193810817BB
:104DD000190748F741E070E060E081EE93E00E943F
:104DE000942AD62E81EE93E00E946B275801FFEFA4
:104DF000AF1ABF0AF70180819181800F911F9A83BA
:104E000089836D2DCE0101960E94761077247A94C5
:104E10007D0CFDEFF71538F2C12C81EE93E00E9476
:104E20006B2745012FEF821A920AF7012081318109
:104E3000A20EB31EBA82A982682FCE0101960E94EB
:104E40007610C3945401CD1440F30E5F1F4F070D2D
:104E5000111DBACF80E0A8CFCF93DF931F92CDB7BB
:104E6000DEB76983DC01ED91FC910280F381E02DD6
:104E700041E050E0BE016F5F7F4F09950F90DF91D9
:104E8000CF910895CF93DF93EC018C859D8597FF9B
:104E900005C082E00E94E72B9D878C878C859D85CD
:104EA000DF91CF91089583E00E94FE2B90E008955A
:104EB00083E00C946D2EFC018485958597FD06C0DA
:104EC00082E00E94972B90E00196089582E00E9474
:104ED000972B90E00895FC018485958597FD05C08A
:104EE0002FEF3FEF35872487089582E00C94E72B5E
:104EF000CF93DF93EC0180913801882331F083E078
:104F00000E94182C1816190634F081E090E09B835B
:104F10008A8380E090E0DF91CF910895EEEFFFE784
:104F20002591349181E02B3F3C4D09F080E00895BC
:104F3000FC0190819E5F908342E450E065E675E05D
:104F400080E80C94C92CFC0181819081913A61F434
:104F5000813209F083C047E050E061E371E080E016
:104F60000E94C92C81E00895913209F077C0833204
:104F700069F482819381B0E0A0E080932D01909349
:104F80002E01A0932F01B0933001ECCF803239F481
:104F900067E070E081E391E00E94EF2CE3CF823282
:104FA00009F78281809338010E948E27E0E0F8E0C3
:104FB000882311F0EEEFFAE08091310190913201F7
:104FC000A0913301B0913401803B9440A105B1051B
:104FD000D9F48091380180FD17C0EE3F8AE0F807D0
:104FE00071F587E797E791838083809160008093D4
:104FF000310488E19BE00FB6F894A8958093600097
:105000000FBE90936000AECF808191818737974724
:1050100009F0A8CFA8958091600088618093600016
:105020008091310480936000EE3F8AE0F80789F0B8
:105030008091FE0A9091FF0A9183808393CF8081B3
:1050400091818737980769F29093FF0A8093FE0A4F
:10505000C8CF1092FF0A1092FE0A84CF80E0089514
:105060002FEF3FEFFC01358724870895E1EEF3E051
:105070001382128288EE93E0A0E0B0E084839583EF
:10508000A683B78385E791E0918380838FEF9FEFBD
:10509000958784870895EF92FF920F931F93CF9384
:1050A000DF937B01FC01C281D38110E000E02097F7
:1050B00091F0E881F9810280F381E02DB701CE0102
:1050C000099597FD06C0080F191F0884D985C02DC2
:1050D000EECF0FEF1FEFC801DF91CF911F910F911E
:1050E000FF90EF9008950F931F93CF93DF938B0161
:1050F000FC01C281D381209771F0E881F98104809D
:10510000F581E02DB801CE010995009731F40884AE
:10511000D985C02DF0CF90E080E0DF91CF911F9135
:105120000F9108950F931F93CF93DF938B01FC0191
:10513000C281D381209771F0E881F9810680F781DF
:10514000E02DB801CE010995080F111D0884D985FD
:10515000C02DF0CFF8011082DF91CF911F910F91F8
:1051600008950F931F93CF93DF938B01FC01C281AE
:10517000D381209771F0E881F9810190F081E02DD1
:10518000B801CE010995811105C00884D985C02DCB
:10519000F0CF80E0DF91CF911F910F910895CF93D1
:1051A000DF93FC01DB01218114968C911497820F0F
:1051B0009927991F08978CF5C281D381209731F5E3
:1051C00073836283908112969C93129713962C930B
:1051D000139715968C911597890F808380E014960C
:1051E0009C9114978917E8F41696CD91DC91179746
:1051F000C80FD11D9881C181D0E0C75CDE4F988374
:1052000091819F5F91838F5FEACFEC0188859985BB
:105210000097D9F7B987A887D5CF80E0DF91CF91E4
:10522000089581E0FBCF8091320481110DC082E0AE
:1052300080933A0484E080933B0410923D041092E2
:105240003C0481E0809332048AE394E00895FB01FA
:1052500001900020E9F73197AF01461B570BDC01A5
:10526000ED91FC910280F381E02D0994EF92FF9281
:105270000F931F93CF93DF938C017B01D0E0C0E0AD
:10528000F701EC0FFD1F6491662361F0D801ED91E9
:10529000FC910190F081E02DC8010995892B11F056
:1052A0002196EECFCE01DF91CF911F910F91FF900C
:1052B000EF900895DC01ED91FC910190F081E02DDB
:1052C000099463E871E00C9427290F931F93CF93FF
:1052D000DF93EC010E9436298C01CE010E946129E6
:1052E000800F911FDF91CF911F910F9108958F92A1
:1052F0009F92AF92BF92EF92FF920F931F93CF9323
:10530000DF93CDB7DEB7A1970FB6F894DEBF0FBE1F
:10531000CDBF7C01FA01CB0119A2223008F42AE0AA
:105320008E010F5D1F4F822E912CB12CA12CBF013D
:10533000A50194010E94FB31F901CA016A300CF504
:10534000605DD8016E938D01232B242B252B79F7DB
:1053500090E080E0109721F0BD01C7010E9427294D
:10536000A1960FB6F894DEBF0FBECDBFDF91CF91EF
:105370001F910F91FF90EF90BF90AF909F908F90F3
:105380000895695CDECFCF92DF92EF92FF920F9388
:105390001F93CF93DF932115310581F4DC01ED914B
:1053A000FC910190F081E02D642FDF91CF911F914E
:1053B0000F91FF90EF90DF90CF9009942A30310544
:1053C00001F52AE077FF1DC06A017B01EC016DE267
:1053D0000E945A298C0144275527BA014C195D09AE
:1053E0006E097F092AE0CE010E947729800F911F64
:1053F000DF91CF911F910F91FF90EF90DF90CF90B1
:105400000895DF91CF911F910F91FF90EF90DF9062
:10541000CF900C9477299A01AB01770F660B770B2D
:105420000C94C3292115310541F4DC01ED91FC9167
:105430000190F081E02D642F09940C9477299A0152
:10544000462F50E070E060E00C94122A9A01AB0104
:1054500070E060E00C94122A0F931F93CF93DF93B8
:10546000EC010E94B403688779878A879B87E8816B
:10547000F9810484F585E02DCE01099597FF15C0CB
:105480000E94B403088519852A853B85601B710B32
:10549000820B930B0C811D812E813F816017710758
:1054A0008207930720F38FEF9FEFDF91CF911F913A
:1054B0000F910895FF920F931F93CF93DF93EC0109
:1054C0008B01F42ECE010E942C2A97FD1DC08D3237
:1054D0009105D1F09C01205331092A303105A0F00B
:1054E000FF2019F08E32910579F00130110551F04D
:1054F0000230110589F48D30910571F05CF4099743
:10550000029750F08FEF9FEFDF91CF911F910F9196
:10551000FF9008958097B1F7E881F9810284F385BF
:10552000E02DCE010995CECFBF92CF92DF92EF92C0
:10553000FF920F931F93CF93DF938C01C42F40E012
:105540000E945A2AFC01C12CD12C760197FD3EC045
:10555000B12C0C2E000CDD0BCE17DF07D9F0ED328D
:10556000F10509F43FC0CF01C0970A9798F4AAE06B
:10557000B0E0A70196010E9432326F01FF0FEE08E2
:10558000FF08C60ED71EE81EF91E80E3C81AD10810
:10559000E108F108D801ED91FC910284F385E02D3A
:1055A000C8010995C8010E942C2AFC01C0970A97DE
:1055B00098F2CE17DF0781F2BB2041F0F094E0941F
:1055C000D094C094C11CD11CE11CF11CC701B601D0
:1055D000DF91CF911F910F91FF90EF90DF90CF90CF
:1055E000BF900895BB24B394D5CF4091410450910E
:1055F000420420913F043091400442175307B4F411
:105600009091E8009570E1F39091E80092FD19C047
:105610008093F100809141049091420401968F7330
:105620009927892B19F48EEF8093E800809141042B
:10563000909142040196909342048093410481E04A
:10564000089580E00895EF92FF920F931F93CF93F8
:10565000DF93F82E192FE62E042F81E0860F880F96
:105660000E94F52A83E00E94F52ACF2DD12FEC0E5F
:10567000FD2EF11CCE15DF05B9F007FF13C0FE01AA
:1056800084910E94F52A182F80E00E94F52A812338
:1056900021968111EFCFDF91CF911F910F91FF9054
:1056A000EF9008958881EDCF81E0F5CF8091D7000C
:1056B00081608093D70080EA8093D80089B58061AB
:1056C00089BD89B5826089BD09B400FEFDCF61E066
:1056D00070E080E090E00E94E5038091D8008F7C2C
:1056E00080618093D8008091E000807F8093E0000B
:1056F0000895CF93DF931F92CDB7DEB71982CE0105
:1057000001960E9498270E941329BE016F5F7F4F68
:105710000E944B2889810F90DF91CF9108952FB778
:10572000FC012083F89467706093E9000895CF939B
:10573000DF931F92CDB7DEB7682FCE0101960E948E
:105740008F2B8091F20099819FBF0F90DF91CF91B5
:105750000895EF92FF920F931F93CF93DF931F92C1
:10576000CDB7DEB790914504992371F157FD2CC058
:105770008A017B01682FCE0101960E948F2B8091B8
:10578000F20090E0081719070CF4C801282FF70160
:1057900044E6215030F0409346043091F1003193BB
:1057A000F8CF009739F02091F200211103C02BE6C9
:1057B0002093E80029812FBF0F90DF91CF911F9197
:1057C0000F91FF90EF9008958FEF9FEFF5CFCF935C
:1057D000DF931F92CDB7DEB741E050E0BE016F5FAF
:1057E0007F4F0E94A92B019731F4898190E00F909F
:1057F000DF91CF9108958FEF9FEFF9CFCF93DF9394
:105800001F92CDB7DEB7682FCE0101960E948F2B75
:105810009091E800892F807295FF04C09091F2006A
:1058200080E4891B99819FBF0F90DF91CF910895EC
:105830005F926F927F928F929F92AF92BF92CF9220
:10584000DF92EF92FF920F931F93CF93DF931F92FC
:10585000CDB7DEB7982E6B01B42E052F809145048D
:10586000811113C08FEF9FEF0F90DF91CF911F91A8
:105870000F91FF90EF90DF90CF90BF90AF909F90EF
:105880008F907F906F905F9008958091430480FF88
:1058900005C08091E00082608093E000EB2CF02E48
:1058A000A12C8AEF882E892D8072682E892D807414
:1058B000582E9AE3792EE114F10419F4AA2009F480
:1058C00057C0892D0E94FE2B182F81110AC08A947F
:1058D000882041F261E070E080E090E00E94E50302
:1058E000EACF8E151F0411F00CF01E2D692DCE018C
:1058F00001960E948F2B8091E80085FD03C089816D
:105900008FBFD9CF812F90E0E81AF90A662029F0DD
:105910001150A0F01092F100FBCFF60197FC0AC0E5
:10592000115050F021912093F100FACF249120934F
:10593000F10031961150D0F7C80ED91EAA2021F0DF
:105940007092E800A12CDBCF8091E80085FD08C0B3
:105950007092E800AA24A394E114F10481F2F2CF3A
:10596000E114F10461F6552051F27092E800C7CFBE
:1059700084E6809347048B2D902F76CF1092E90018
:1059800010924204109241049093400480933F048B
:105990000895DF92EF92FF920F931F93CF93DF93BF
:1059A000D82E8A01EB017B01E40EF51ECE15DF0532
:1059B00059F0D7FE12C0FE0184910E94F52A21966B
:1059C0008111F4CF0FEF1FEFC801DF91CF911F912D
:1059D0000F91FF90EF90DF9008958881EECFCF93E5
:1059E000DF93EC019B01B4E6ABEF21153105F1F03B
:1059F000A9012134310514F040E450E08091E80021
:105A000082FFFCCF942FFB01E21BF30BEC0FFD1F79
:105A1000915028F08091F10080833196F9CFB093B6
:105A20004604A093E800241B350BDFCFCB01DF91A8
:105A3000CF9108951F920F920FB60F921124CF921B
:105A4000DF92FF920F931F932F933F934F935F9398
:105A50006F937F938F939F93AF93BF93EF93FF9336
:105A6000CF93DF93CDB7DEB76C97DEBFCDBF10927B
:105A7000E9008091E80083FF2FC089E0FE01759660
:105A8000FE2E0F2F815029F09091F10090833196D6
:105A9000F9CF84E68093460482EF8093E8008D89F5
:105AA00087FF38C09091E80090FFFCCF982F907648
:105AB00009F000C19E894F89588D2F89188D911149
:105AC00030C0803859F5809144048093F1001092E1
:105AD000F1008EEF8093E8006C960FB6F894DEBF6D
:105AE0000FBECDBFDF91CF91FF91EF91BF91AF91ED
:105AF0009F918F917F916F915F914F913F912F91E6
:105B00001F910F91FF90DF90CF900F900FBE0F90DD
:105B10001F9018959EEF9093E800C8CF1092F10067
:105B2000D6CF913059F48111D4CF4130510589F647
:105B3000809144048D7F80934404CBCF933049F40B
:105B40008111C7CF4130510521F680914404826014
:105B5000F2CF953041F48091E80080FFFCCF2068BF
:105B60002093E300B6CF963009F076C0CB8CDC8C66
:105B7000123039F590E080E00E94BE2C0E94792B13
:105B80001F8299E099831A8391E09E8390EA988717
:105B90009CE099872091410430914204275F3F4F58
:105BA0003C832B838D83C6010E94BE2C49E050E0CC
:105BB000BE016F5F7F4F80E00E94C92C0E94792B4D
:105BC00088CFC6010E94BE2C0E9413296F2D702F12
:105BD0000E947328009731F00CF07BCF81E2809314
:105BE000EB007ACF113061F11330C1F78F89882330
:105BF00081F1823049F440E866E084EC95E00E944F
:105C0000232B882359F365CF813029F440E86AE0DB
:105C100089EB95E0F4CF833009F70E9413298E01B8
:105C20000F5F1F4FB8010E949228F80101900020D9
:105C3000E9F73197BF01601B710B40E0C801DFCF6E
:105C400067EA75E0FB01449150E080E80E94C92CAE
:105C500040CF6BEC75E0F6CF973009F4BFCF9830AA
:105C600021F481E08093F10034CF993009F031CFF5
:105C7000837009F0B3CFEAE3F1E081E031E096E32D
:105C80002191222371F08093E9003093EB00DF0132
:105C900011972C912093EC009093ED008F5F87304B
:105CA00079F78EE78093EA001092EA008F8980935B
:105CB00045040FCF8B8D9C8D0E94BE2C898D811148
:105CC00005C08F2D902F0E94A3279BCF0E941329E0
:105CD0006F2D702F0E94B12894CF8093E90080919E
:105CE000F200882319F08AE38093E80008951F9258
:105CF0000F920FB60F9211242F933F934F935F9300
:105D00006F937F938F939F93AF93BF93CF93EF93B3
:105D1000FF93C091E1008091E100837F8093E100D7
:105D2000C3FF0FC01092E90081E08093EB00109256
:105D3000EC0082E38093ED001092450488E08093AC
:105D4000F000C2FF15C083E00E946D2E80914704D1
:105D5000882329F0809147048150809347048091E3
:105D60004604882329F0809146048150809346049C
:105D7000C4FF23C08091E2008E7E81608093E200A8
:105D80008091E1008F7E8093E100809143048E7EBC
:105D9000806180934304FF91EF91CF91BF91AF91C8
:105DA0009F918F917F916F915F914F913F912F9133
:105DB0000F900FBE0F901F901895C0FFECCF8091F1
:105DC000E2008E7E80618093E2008091E1008E7E11
:105DD0008093E100809143048E7E8160DACF10923F
:105DE000450410924404109243040E94562BE1EEA5
:105DF000F0E080818E7E80838DE08093E200559A72
:105E0000209A08958091E0008D7F8093E00080913A
:105E1000E00081FD11C08091430480FF0DC080919E
:105E2000440481FF09C00E94562B8091E0008260EB
:105E30008093E00081E0089580E008950895109235
:105E4000A9041092AA040895CF93DF93CDB7DEB7CB
:105E500069970FB6F894DEBF0FBECDBFFC01DB0122
:105E60008C918F5F8C939E012D5F3F4F8DE0D90108
:105E70001D928A95E9F729E0298384E08A8391E0DD
:105E80009D8383E08E832A8721E22B879C879D87D1
:105E90009F8722E2288B27E02B8B25E02C8B8E8B93
:105EA00020E430E0388F2F8B998F82818B8395850A
:105EB0008685998B8A8B838180688D8B49E150E040
:105EC000BE016F5F7F4F80E00E94C92C69960FB6BC
:105ED000F894DEBF0FBECDBFDF91CF910895EF9252
:105EE000FF920F931F93CF93DF93FB012081213803
:105EF000A1F52381223289F5DC0112964C9124818F
:105F000035814217130649F5EC0181E00E94D23138
:105F10000B851C85F12CE12C0115110589F0F80188
:105F2000448155816281738180E80E94C92C8F3F32
:105F3000980761F0E80EF91ED8010D911C91ECCF85
:105F400081E08F8780E00E94D231C701DF91CF913D
:105F50001F910F91FF90EF90089590E080E0F6CFB1
:105F6000CF93DF93EC01DB012A8114968D919C91F4
:105F700015972817190659F411968C9111979C9131
:105F8000913A39F4982F9D7F81E0913051F080E073
:105F900008C09132E1F78B3039F412968C918F87DB
:105FA00081E0DF91CF9108958A3021F413968C918E
:105FB000888BF6CF893059F716968D919C91823057
:105FC000910539F462E070E0CE0141960E94EF2C19
:105FD000DECF0197E1F661E070E0CE0142960E94CB
:105FE000EF2C198AD4CFFC01A385B485109771F4E6
:105FF0007487638785859685DB0114962D913C9186
:10600000820F931F968785870895DC018D919C915F
:1060100011970097D1F76D937C93ECCFAF92BF921D
:10602000CF92DF92EF92FF920F931F93CF93DF9364
:106030001F92CDB7DEB77C0169836A01590141E047
:1060400050E0BE016F5F7F4FFC0183810E94182CDE
:106050008C0197FD0BC0F7018381A501B601806417
:106060000E94182C080F191F97FD8C01C8010F9072
:10607000DF91CF911F910F91FF90EF90DF90CF9024
:10608000BF90AF900895CF92DF92EF92FF921F934F
:10609000CF93DF93162F7A0169010E940E30EC0135
:1060A000E0916002F0916102309729F09C01A60115
:1060B000B701812F0995CE01DF91CF911F91FF90FC
:1060C000EF90DF90CF900895CF93DF93EC0181E0C4
:1060D0008C838D839E01265F3F4F3F832E831986DD
:1060E00018862AE831E0398328831C861B861E86A1
:1060F0001D868F87888B198A1A8A81EC8A870E946D
:106100001329BE01DF91CF910C94CF288091AB046D
:10611000811107C083EB94E00E94643081E080939A
:10612000AB0483EB94E00895FC0115828091CC04CC
:10613000811113C01092D5041092D4048FEC95E015
:106140009093D7048093D6048AE390E09093D90487
:106150008093D80481E08093CC040E94863064ED63
:1061600074E00C94F32F0F93FC016183428323832B
:1061700004830F91089525E0FC0111922A95E9F717
:106180000895FC019081692B60830895CF93DF937C
:10619000EC010E94863025E030E0AE0161E0DF9145
:1061A000CF910C944330CF93DF93EC0198818D8194
:1061B00098130CC08981811109C08A81811106C0A0
:1061C0008B81811103C08C81882329F0CE010E942C
:1061D000C63088818D83DF91CF910895CF93DF936F
:1061E000EC010E94BB30CE01DF91CF910C94D330F3
:1061F0000C94EE3086EC94E00C949430CF93DF93C3
:10620000CDB7DEB769970FB6F894DEBF0FBECDBF2E
:10621000FC01DB019C919F5F9C939E012D5F3F4F92
:1062200081E1D9011D928A95E9F729E0298384E06B
:106230008A8391E09D8383E08E832A8721E22B87E6
:106240009C879D879F8722E2288B25E3298B27E067
:106250002B8B25E02C8B8E8B20E430E0388F2F8B1E
:10626000998F82818B83838180688D8B49E150E097
:10627000BE016F5F7F4F80E00E94C92C69960FB608
:10628000F894DEBF0FBECDBFDF91CF9108950F937D
:106290001F93CF93DF93EB018A01FC01838180641C
:1062A0000E94182CE0916002F0916102309749F051
:1062B0009C01A801BE0187E0DF91CF911F910F9152
:1062C0000994DF91CF911F910F9108950A970C9433
:1062D0004731DC01FB0112962C9112978481958144
:1062E0002817190641F491818081813A31F49D7F0C
:1062F00081E0913009F080E008958132E1F79B3030
:1063000029F4828152968C9381E008959A3099F70E
:10631000828153968C93F8CFFB0120812138B1F410
:106320002381223299F4DC0112964C911297248138
:1063300035814217130651F421E052962C9345E320
:1063400050E069E076E080E80C94C92C90E080E0B1
:106350000895CF93DF93EC0181E08C838D839E01C0
:106360002F5E3F4F3F832E83198618861D861C861D
:106370001F861E86188A26E931E03983288324EA9D
:1063800031E03B872A878A8B8B8B81EC898B0E943B
:106390001329BE01DF91CF910C94CF288AED94E0B0
:1063A0000C94A9310895AA1BBB1B51E107C0AA1F79
:1063B000BB1FA617B70710F0A61BB70B881F991FA6
:1063C0005A95A9F780959095BC01CD01089597FB4A
:1063D000072E16F4009407D077FD09D00E94D33120
:1063E00007FC05D03EF4909581959F4F08957095D8
:1063F00061957F4F0895A1E21A2EAA1BBB1BFD01D8
:106400000DC0AA1FBB1FEE1FFF1FA217B307E40793
:10641000F50720F0A21BB30BE40BF50B661F771FEB
:10642000881F991F1A9469F76095709580959095CB
:106430009B01AC01BD01CF010895EE0FFF1F059038
:10644000F491E02D0994A29FB001B39FC001A39FD6
:10645000700D811D1124911DB29F700D811D11249D
:10646000911D08950E942332A59F900DB49F900D19
:10647000A49F800D911D112408950024A7FD009470
:106480002A0F301D401D501D601D701D801D901D68
:1064900008950024A7FD00942A17300540055005F3
:1064A00060057005800590050895FB01DC0102C0C0
:1064B00005900D9241505040D8F70895FB01DC0142
:1064C0008D91059080190110D9F3990B0895FB0166
:1064D000DC014150504030F08D910590801919F445
:1064E0000020B9F7881B990B0895FB01DC0104C05B
:1064F0008D910190801921F441505040C8F7881BBC
:10650000990B0895FB01DC0102C001900D924150EE
:106510005040D8F708956817790768F4FB01DC014B
:10652000E40FF51FA40FB51F02C002900E92415058
:106530005040D8F708950C948232F999FECF92BD5D
:1065400081BDF89A992780B50895262FF999FECF35
:106550001FBA92BD81BD20BD0FB6F894FA9AF99A80
:0A6560000FBE01960895F894FFCFD6
:10656A0003FF6D0B01290032000140000101000107
:10657A007F02C409FA00FFFFFFFF000000000000CD
:10658A0000000000000000000000FFC800FFFFFF3D
:10659A00FF00E100000000000000C180810000004F
:1065AA00FFFFFFFFFFFFFFFFFFFFFFFF6174726541
:1065BA00757300AF01F7C26766363597969495935F
:1065CA0092F6F5F4F100000000510DE90C340DE2E9
:1065DA000C000000002C277827532758275B276BCD
:1065EA002742270D0A0000000000B02F242F6F2F2A
:1065FA008004000000006931FE308C31E20C473122
:06660A00F6FF00006631FE
:00000001FF
